:020000040800F2
:1000000000040020671A0008590900085B0900086D
:100010005F09000863090008670900080000000084
:100020000000000000000000000000006B09000854
:100030006D090008000000006F0900087109000840
:10004000C7060008871A0008871A0008871A0008E0
:10005000871A0008871A0008871A0008871A0008FC
:10006000871A0008871A0008871A0008871A0008EC
:10007000871A0008871A0008871A0008871A0008DC
:10008000871A0008871A0008871A0008871A0008CC
:10009000871A0008871A0008871A0008871A0008BC
:1000A000871A0008871A0008871A0008871A0008AC
:1000B000871A0008871A0008871A0008871A00089C
:1000C000871A0008871A0008871A0008871A00088C
:1000D000871A0008871A0008871A0008871A00087C
:1000E000871A0008871A0008871A0008871A00086C
:1000F000871A0008871A0008871A0008871A00085C
:10010000871A0008871A0008871A0008871A00084B
:10011000871A0008871A0008871A0008871A00083B
:10012000871A0008871A0008871A0008871A00082B
:1001300000F002F800F03CF80AA090E8000C8244BD
:100140008344AAF10107DA4501D100F031F8AFF29A
:10015000090EBAE80F0013F0010F18BFFB1A43F0A5
:10016000010318473024000050240000103A24BF37
:1001700078C878C1FAD8520724BF30C830C144BF0C
:1001800004680C607047000000230024002500264E
:10019000103A28BF78C1FBD8520728BF30C148BFEA
:1001A0000B6070471FB5AFF300801FBD10B510BDC9
:1001B00001F081FC1146FFF7F5FF00F073FB01F041
:1001C0009FFCFFF7F3FF01F0A5FC0000002904DA13
:1001D0004A4211B22D22027001E0202202706422F4
:1001E00091FBF2F23032D3B2421C104613706422FB
:1001F00091FBF2F302FB131211B20A2291FBF2F20D
:100200003032D3B2421C104613700A2291FBF2F333
:1002100002FB131211B201F13002D3B2421C10469C
:100220001370704708B54020ADF8000003208DF82A
:10023000020014208DF803006946FF4801F046F8DB
:100240008020ADF8000003208DF8020014208DF806
:1002500003006946F84801F039F808BD1E2001E0A6
:10026000411EC8B20028FBD1704741F2883000E03F
:10027000401E0028FCD1704700B58020EE491031A7
:1002800008604020ED49C1F8100CFFF7E7FFEA488D
:100290000830006808B9012000E0002010F0800F4D
:1002A00001D0002000BD8020E34914310860FFF731
:1002B000D5FFE248D0F8080C10F0800F01D00020E4
:1002C000F0E78020DC4914310860FFF7C7FF012008
:1002D000E8E700B54020D84914310860FFF7BEFFB9
:1002E0008020D649C1F8140CFFF7B8FF4020D2494E
:1002F00010310860FFF7B2FF8020D049C1F8100C20
:10030000FFF7ACFF00BD00B54020CB4914310860B9
:10031000FFF7A4FF8020C949C1F8140CFFF79EFF26
:100320004020C54910310860FFF798FF4020C349BD
:10033000C1F8140CFFF792FF00BD00B54020BE4984
:1003400014310860FFF78AFF8020BC49C1F8100C07
:10035000FFF784FF4020B84910310860FFF77EFFA7
:100360004020B649C1F8140CFFF778FF00BD00B576
:100370004020B14914310860FFF770FF8020AF4979
:10038000C1F8100CFFF76AFF4020AB49103108603C
:10039000FFF764FFA948D0F8080C10F0800F07D0D1
:1003A0004020A54914310860FFF758FF002000BD28
:1003B0004020A14914310860FFF750FF0120F6E703
:1003C00000B5034608221BE040209B491431086019
:1003D000FFF744FF13F0800F04D0802096491031BE
:1003E000086003E080209449143108605806030E29
:1003F000FFF734FF4020904910310860FFF72EFFCF
:100400001000A2F10101CAB2DED140208A491431A4
:10041000086000BD00B50822002380208649103105
:10042000086015E05806030E402083491431086027
:10043000FFF714FF40208149C1F8100CFFF70EFFB1
:100440007D480830006810F0800F01D043F00103B0
:100450001000A2F10101CAB2E4D140207649143162
:100460000860184600BD70B504460D461646FFF7F5
:1004700003FF08B9002070BD2046FFF7A1FFFFF77A
:1004800076FF18B9FFF725FF0020F4E72846FFF7AD
:1004900097FFFFF76CFF3046FFF792FFFFF767FF0C
:1004A000FFF717FFFFF7E1FE0120E4E770B5044610
:1004B0000D46FFF7E1FE08B9002070BD2046FFF7AA
:1004C0007FFFFFF754FF30B9FFF703FF01205C49BE
:1004D00008700020F1E72846FFF772FFFFF747FF9B
:1004E000FFF7CAFE601CC0B2FFF76AFFFFF73FFFCD
:1004F000FFF790FF0646FFF720FFFFF7EAFE3046C2
:10050000DBE710B500F036FA4FF4803000F052FA15
:1005100000F08FFA4B49087008460078012826D170
:10052000002000F0C5FA002000F0D2FA4FF48060FD
:1005300000F0C6FA022000F0FDFF102001F00DF8D7
:100540004FF4E0114FF4803000F097FA012000F0F2
:100550009FFA00BF392000F050FA0028FAD002209C
:1005600000F099FA00BF00F09EFA0828FBD10121A3
:100570000C2000F065FB0121302000F061FB01211F
:10058000C02000F05DFB012140F2011000F058FB9B
:1005900010BD08B501213C2000F052FB4FF4007063
:1005A000ADF8000018208DF8030003208DF802003C
:1005B0006946254800F08AFE4FF48060ADF80000DF
:1005C00004208DF8030069461F4800F07FFE08BD37
:1005D00000B587B001214FF4904000F031FB0020BE
:1005E000ADF80400ADF806004FF40070ADF8080057
:1005F0000020ADF80A0001A9144800F020FC4FF4D7
:10060000E13003900020ADF81000ADF81200ADF815
:100610001400ADF818000C20ADF8160003A90B4823
:1006200000F0B3FB40F22551084800F0F1FC012234
:1006300040F2255105480BE0000C0140000001404C
:1006400000000020060000200008014000380140A2
:1006500000F017FC0121B34800F007FC07B000BD13
:1006600008B54FF4E06000F061FD00208DF8000057
:100670008DF80100684600F05EFD08BD10B501214F
:10068000C80200F0EAFA4FF4C07000F018FD4120F3
:1006900000F01FFD502000F032FD00F03BFD00F0A7
:1006A00024FD10BD00E0401E0028FCD1704707E08B
:1006B000002100E0491C4CF250329142FAD3401E16
:1006C0000028F5D1704710B5502000F012FD00F061
:1006D00021FD10BD10B504462146924800F034FCBF
:1006E0000120FFF7E4FF10BD00B580223E21D0209D
:1006F000FFF7B9FE07221521D020FFF7B4FE1E2216
:100700001621D020FFF7AFFE00221721D020FFF7DF
:10071000AAFE00223E21D020FFF7A5FE00BD00B5B5
:1007200087B01E21D020FFF7C1FE7F4908701D2130
:10073000D020FFF7BBFE7C49487008460078497816
:1007400040EA012000B2794908800846B0F900006B
:1007500001F026FDCDE9040175A00CC8049801F054
:10076000D1FACDE9020101F0CDFC00B26F49088059
:100770002021D020FFF79AFE6B4988701F21D020DE
:10078000FFF794FE6849C87008468078C97840EA47
:10079000012000B2684908800846B0F9000001F065
:1007A000FFFCCDE9040162A00CC8049801F0AAFA8C
:1007B000CDE9020101F0A6FC00B25F4908802221C8
:1007C000D020FFF773FE584908712121D020FFF790
:1007D0006DFE5549487108460079497940EA012083
:1007E00000B2564908800846B0F9000001F0D8FC74
:1007F000CDE904014EA00CC8049801F083FACDE9BC
:10080000020101F07FFC00B24C4908801C21D0207D
:10081000FFF74CFE444988711B21D020FFF746FEAC
:100820004149C87108468079C97940EA012000B27F
:10083000434908800846B0F9000043F2903108446B
:1008400001F0AEFCCDE904013EA00CC8049801F013
:1008500059FACDE902013DA00CC8029801F066F9F1
:10086000CDE9000101F04EFC00B23549088007B027
:1008700000BD70B505462846FFF72CFF3A20FFF76C
:1008800029FF002405E03349085DFFF723FF601CC2
:10089000C4B2042CF7DB2020FFF71CFF2020FFF759
:1008A00019FF70BD10B5FFF72CFEFFF772FEFFF7C2
:1008B0008FFEFFF7B7FC0A20FFF7F9FEFFF714FFE2
:1008C0002EE0FFF72CFF1948B0F900102148FFF780
:1008D0007DFC5820FFF7CDFF1748B0F900101D48E8
:1008E000FFF774FC5920FFF7C4FF1448B0F900105B
:1008F0001848FFF76BFC5A20FFF7BBFF1048B0F910
:1009000000101448FFF762FC5420FFF7B2FF0D20DF
:10091000FFF7E0FE0A20FFF7DDFE0520FFF7C7FE28
:10092000CFE7000000380140280000200C00002024
:100930000000000000C02C400E000020100000202D
:100940001200002000000000008071400000000044
:100950000080414007000020704700BFFEE700BF55
:10096000FEE700BFFEE700BFFEE770477047704735
:1009700070470000DB48006840F00100D94908607A
:1009800008464068D8490840D6494860084600688B
:10099000D6490840D34908600846006820F4802002
:1009A00008600846406820F4FE0048604FF41F00CD
:1009B00088607047CB49096821F48031C94A1160C9
:1009C0001146096821F480211160B0F5803F03D001
:1009D000B0F5802F0ED106E0C249096841F480319C
:1009E000C04A116007E0BF49096841F4A021BD4A2F
:1009F000116000E000BF00BF704710B50146002243
:100A0000002300204A11012A02D1B64C236806E0D7
:100A1000022A02D1B34C236A01E0B24C636A01F0AE
:100A20001F02012494401C4201D0012000E000205C
:100A300010BD70B500240025002600BF3120FFF74F
:100A4000DCFF0646641CB4F5A06F01D0002EF5D083
:100A50003120FFF7D2FF08B1012500E0002528462C
:100A600070BD00219F4A116821F0F80141EAC001E0
:100A7000116070479E49086070470022994B5A6880
:100A800022F47C1240EA01031A43964B5A607047E5
:100A90009749086670470021924A516821F0030186
:100AA0000143516070478F48406800F00C00704768
:100AB00000218C4A516821F0F001014351607047D8
:100AC0000021884A516821F4E06101435160704778
:100AD0000021844A516821F4605141EAC00151600B
:100AE000704729B17F4A527A02437E4B5A7206E020
:100AF0007C4A527AC343DBB21A407A4B5A7270472F
:100B00007B49D831086070470021764A516821F44A
:100B100040410143516070470021724A20321170F8
:100B2000704A82F82010012802D004280AD104E07B
:100B300001216C4A2032117005E00521694A2032FA
:100B4000117000E000BF00BF70476A49086070473D
:100B50006449096A0143634A11627047654944392F
:100B60000860704730B500210022002300245D4D4D
:100B70006D6805F00C0121B1042905D0082923D1A5
:100B800005E05D4D056022E05B4D05601FE0554DC1
:100B90006D6805F47012534D6D6805F480330225BD
:100BA00005EB92421BB9554D554305600BE04D4D89
:100BB0006D6815F4003F03D0504D5543056002E0C9
:100BC0004D4D5543056002E04B4D056000BF00BF31
:100BD000444D6D6805F0F0010909494D6C5C0568EC
:100BE000E54045603F4D6D6805F4E061090A444DFC
:100BF0006C5C4568E54085603A4D6D6805F4605170
:100C0000C90A3F4D6C5C4568E540C560354D6D686F
:100C100005F44041890B3A4D10356C5CC568B5FB55
:100C2000F4F5056130BD29B12E4A526902432D4BBE
:100C30005A6104E02B4A526982432A4B5A61704739
:100C400029B1284A92690243264B9A6104E0254A59
:100C500092698243234B9A61704729B1214AD26934
:100C60000243204BDA6104E01E4AD26982431D4BE5
:100C7000DA61704729B11B4AD2680243194BDA6026
:100C800004E0184AD2688243164BDA60704729B1F3
:100C9000144A12690243134B1A6104E0114A1269A3
:100CA0008243104B1A6170471249403908607047FF
:100CB0000F49C86470470B49C87170470948406ABA
:100CC00040F0807007494862704701460020054A9D
:100CD00092680A4201D0012000E0002070470149DB
:100CE00088727047001002400000FFF8FFFFF6FE18
:100CF000000042428004424200127A0000093D0096
:100D00001400002010B50446E248844209D10121B4
:100D10008803FFF7AFFF00214FF48040FFF7AAFFE1
:100D200032E0DD48844209D101214804FFF7AFFFDA
:100D300000214FF40030FFF7AAFF25E0D748844296
:100D400009D101218804FFF7A2FF00214FF4802080
:100D5000FFF79DFF18E0D248844209D10121C80461
:100D6000FFF795FF00214FF40020FFF790FF0BE005
:100D7000CC48844208D101210805FFF788FF0021F3
:100D80004FF48010FFF783FF10BD2DE9F04786B0C8
:100D900004460D460026002700BF00BFB246A889C2
:100DA00000B100BFA246268A4CF6FF700640E888D4
:100DB00006432682A6894EF6F3100640A8882989A4
:100DC0000843698908430643A681A68A4FF6FF4077
:100DD0000640A8890643A68201A8FFF7C3FE544631
:100DE000AC48824501D1049F00E0039F07EBC70098
:100DF00000EB071029688900B0FBF1F86420B8FB0C
:100E0000F0F006013009642101FB1089322101EB69
:100E100009106421B0FBF1F000F00F0006432681B9
:100E200006B0BDE8F0874FF41651016000218180C3
:100E3000C18001810C21418100218181704710B561
:100E40000022028A4FF2FF031A400B884C8823438A
:100E50008C882343CC8823431A43028210BD00218F
:100E6000018041808180C180704721B1828942F434
:100E70000052828104E082894DF6FF731A4082811C
:100E80007047F0B50024002500260023A1F5106767
:100E90006A3F00D100BF0346C1F3421401F01F05B1
:100EA000012707FA05F6012C01D10C3304E0022CCE
:100EB00001D1103300E014331AB11F6837431F60AB
:100EC00002E01F68B7431F60F0BD10B51AB1838AF6
:100ED0000B43838204E0838ACC43A4B22340838201
:100EE00010BD028A4FF6F0731A400282028A0A434A
:100EF0000282704782894FF2FF731A408281828991
:100F00000A438281704721B1828942F002028281C4
:100F100004E082894FF6FD731A4082817047028A8D
:100F20004FF6DF731A400282028A0A430282704738
:100F300021B1028A42F48042028204E0028A4BF626
:100F4000FF731A4002827047C1F308028280704723
:100F500001468888C0F308007047818941F001018B
:100F600081817047028BD2B20283028B42EA012256
:100F700002837047028B02F47F420283028B0A4392
:100F80000283704721B1828A42F02002828204E00B
:100F9000828A4FF6DF731A408282704721B1828ABB
:100FA00042F01002828204E0828A4FF6EF731A4008
:100FB0008282704721B1828A42F00802828204E074
:100FC000828A4FF6F7731A4082827047828A4FF600
:100FD000FB731A408282828A0A438282704721B15F
:100FE000828A42F00202828204E0828A4FF6FD7316
:100FF0001A408282704702460020B1F5007F00D17E
:1010000000BF13880B4201D0012000E00020704790
:1010100001F40072B2F5007F00D100BFCA43028024
:10102000704770B502460023002400250020A1F57A
:1010300010666A3E00D100BFC1F3421501F01F04E3
:10104000012606FA04F4012D02D19689344006E007
:10105000022D02D1168A344001E0968A34400B12E8
:10106000012606FA03F31688334014B10BB10120B0
:1010700000E0002070BD10B500220023A1F510642F
:101080006A3C00D100BF0A1201249440A3B2DC43A1
:10109000048010BD0038014000440040004800407A
:1010A000004C00400050004010B50121C802FFF77D
:1010B000EEFD00214FF40060FFF7E9FD10BD0021B7
:1010C000174A126822F4C0710143164AC2F8041C80
:1010D00070470021124A126822F07F0100F07F025F
:1010E0001143104AC2F8041C704701200E490860E1
:1010F000704700F07F010A4A121F1160704740F0EC
:101100008001074A121F116070470548001D0068E2
:10111000C0B2704700200249091D086070470000F6
:10112000042C004000200040A480054232490143C5
:10113000324A1160704770B5002100230F22C47835
:101140000CB32E4C246804F4E064C4F5E064210A76
:10115000C1F10403CA40447804FA03F184781440CE
:1011600021430901264C0678A155047804F01F0597
:101170000124AC4005786D114FF0E02606EB8505A3
:10118000C5F8004109E0047804F01F040125A540DA
:101190001C4C0678761144F8265070BD1A4A0A4055
:1011A0000243164B1B1F1A60704741B1134A121DB0
:1011B000126802434FF0E023C3F8102D07E00F4AF6
:1011C000121D126882434FF0E023C3F8102D7047C0
:1011D000042808D14FF0E021096941F004014FF0E3
:1011E000E022116107E04FF0E021096921F00401DC
:1011F0004FF0E022116170470000FA050CED00E0AD
:1012000000E400E080E100E080FFFF1F10B504462D
:10121000BF48844208D101210420FFF72BFD0021A3
:101220000420FFF727FD46E0BA48844208D1012197
:101230000820FFF71FFD00210820FFF71BFD3AE003
:10124000B548844208D101211020FFF713FD002189
:101250001020FFF70FFD2EE0B048844208D1012195
:101260002020FFF707FD00212020FFF703FD22E0EB
:10127000AB48844208D101214020FFF7FBFC00214C
:101280004020FFF7F7FC16E0A648844208D1012170
:101290008020FFF7EFFC00218020FFF7EBFC0AE045
:1012A000A148844207D101218015FFF7E3FC00210A
:1012B000A015FFF7DFFC10BD10B501210846FFF7B0
:1012C000D9FC00210120FFF7D5FC10BDF0B50022AC
:1012D0000023002400250026002791F803C00CF00D
:1012E0000F0291F803C01CF0100F03D091F802C058
:1012F0004CEA0202B1F800C01CF0FF0F31D00668C2
:1013000000242BE04FF0010C0CFA04F5B1F800C0FA
:101310000CEA0503AB4220D1A5004FF00F0C0CFAEC
:1013200005F7BE4302FA05FC4CEA060691F803C035
:10133000BCF1280F06D14FF0010C0CFA04FCC0F8E8
:1013400014C00AE091F803C0BCF1480F05D14FF07A
:10135000010C0CFA04FCC0F810C0641C082CD1D39A
:101360000660B1F800C0BCF1FF0F34DD4668002410
:101370002EE004F1080C4FF0010E0EFA0CF5B1F856
:1013800000C00CEA0503AB4221D1A5004FF00F0CC1
:101390000CFA05F7BE4302FA05FC4CEA060691F882
:1013A00003C0BCF1280F05D104F1080C0EFA0CFEA5
:1013B000C0F814E091F803C0BCF1480F07D104F164
:1013C000080C4FF0010E0EFA0CFEC0F810E0641C81
:1013D000082CCED34660F0BD4FF6FF71018002218C
:1013E00081700421C17070470246002093680B424F
:1013F00001D0012000E0002070470146886880B2DB
:10140000704702460020D3680B4201D0012000E063
:10141000002070470146C86880B27047016170477C
:10142000416170470AB1016100E041617047C160EC
:1014300070474FF480320A43826181618261826920
:10144000826970470022394B1A684FF680731A4040
:1014500042EA00120A43354B1A6070473449C861AA
:101460007047F0B500220023002500242F4E756838
:10147000C0F3034482B200F44016B6F5401F08D111
:1014800025F07065294E766826F07066274F7E60DD
:1014900012E000F48016B6F5801F06D1032606FA86
:1014A00004F39D4345F0706506E0460D360102FAEF
:1014B00006F6B54345F0706521B1460D360102FAD6
:1014C00006F63543194E7560F0BD30B500228B0726
:1014D0001C0F0F2303FA04F2144B08338C1053F83B
:1014E000244094438D1043F825408C1053F8243049
:1014F0008C07240F00FA04F423430C4C08348D109D
:1015000044F8253030BD0A49DC31086070470000DE
:1015100000080140000C014000100140001401408F
:1015200000180140001C0140002001400000014063
:10153000000020420021FC4A116801F038010143FB
:1015400011607047F849096821F00801F64A1160F6
:1015500011460968014311607047F349096821F099
:101560001001F14A1160114609680143116070478A
:10157000EE48ED494860EE4848607047EA48006927
:1015800040F08000E849086170470420E649C968D6
:1015900001F00101012901D101200EE0E249C968F1
:1015A00011F0040F01D0022007E0DF49C96811F0F3
:1015B000100F01D0032000E0042070470020FF201E
:1015C00000E0401E0028FCD1704770B50446042599
:1015D000FFF7DBFF054605E0FFF7F0FFFFF7D5FF5C
:1015E0000546641E012D01D1002CF5D104B9052555
:1015F000284670BD70B50446042540F6FF70FFF71D
:10160000E4FF0546042D19D1C748006940F00200E7
:10161000C549086108464461006940F0400008611E
:1016200040F6FF70FFF7D1FF0546052D06D0BE48F6
:10163000006941F6FD710840BB490861284670BD4C
:1016400010B5042440F6FF70FFF7BFFF0446042CDA
:1016500018D1B548006940F00400B3490861084654
:10166000006940F04000086140F6FF70FFF7ADFFF1
:101670000446052C06D0AC48006941F6FB710840D1
:10168000A9490861204610BD10B5042440F6FF703A
:10169000FFF79BFF0446042C3BD1A448A249886075
:1016A000A34888600846006940F0200008610846A9
:1016B000006940F04000086140F6FF70FFF785FFC9
:1016C0000446042C1CD19848006941F6DF7108409B
:1016D000954908610846006940F010000861A5209E
:1016E000944908800F20FFF770FF0446052C10D0A6
:1016F0008D48006941F6EF7108408B49086108E0A8
:10170000052C06D08848006941F6EF7108408649EB
:101710000861204610BD2DE9F04104460D4604261F
:1017200000270F20FFF751FF0646042E26D17E48E2
:10173000006940F001007C49086125800F20FFF717
:1017400044FF0646042E10D1A71C280C38800F2019
:10175000FFF73BFF0646052E10D07348006941F69F
:10176000FE7108407049086108E0052E06D06E48F9
:10177000006941F6FE7108406B4908613046BDE8DA
:10178000F08170B504460D4604260F20FFF71DFFBB
:101790000646042E13D16448006940F001006249F6
:1017A000086125800F20FFF710FF0646052E06D0A2
:1017B0005D48006941F6FE7108405B4908613046AA
:1017C00070BD70B504460D4604260F20FFF7FDFEE0
:1017D0000646042E17D155485349886054488860FE
:1017E0000846006940F01000086125800F20FFF7CF
:1017F000ECFE0646052E06D04B48006941F6EF7117
:10180000084049490861304670BD2DE9F04704465B
:101810004FF6FF752E462F46A8464FF00409E443C5
:10182000E5B2C4F30726C4F307474FEA14680F2054
:10183000FFF7CBFE8146B9F1040F41D13B483A494D
:1018400088603B4888600846006940F010000861E5
:10185000FF2D06D03748083005800F20FFF7B5FE72
:101860008146B9F1040F08D1FF2E06D031480A3065
:1018700006800F20FFF7A9FE8146B9F1040F08D1B9
:10188000FF2F06D02B480C3007800F20FFF79DFE5E
:101890008146B9F1040F09D1B8F1FF0F06D02648EF
:1018A000A0F80E880F20FFF790FE8146B9F1050FD2
:1018B00006D01D48006941F6EF7108401A490861D9
:1018C0004846BDE8F08770B50446042540F6FF7031
:1018D000FFF77BFE0546042D4BD114481249886062
:1018E000134888600846006940F0200008610846F7
:1018F000006940F04000086140F6FF70FFF765FEA8
:101900000546042D2CD10848006941F6DF710840D6
:10191000054908610846006940F0100008616CB193
:101920000020044908800CE00020024023016745A4
:10193000AB89EFCD00F8FF1F00F0FF1FA520454940
:10194000088040F6FF70FFF740FE0546052D10D0D9
:101950004148006941F6EF7108403F49086108E0DD
:10196000052D06D03C48006941F6DF7108403A4930
:101970000861284670BD2DE9F04104460D46164623
:101980000427364834498860354888600F20FFF7BF
:101990001CFE0746042F19D12F48006940F01000A3
:1019A0002D49086146F0F800284320432949891C45
:1019B00008800F20FFF709FE0746052F06D02648AE
:1019C000006941F6EF710840234908613846BDE8D7
:1019D000F0812148C069800870471F48006A70473D
:1019E00000201D49C96911F0020F01D0012000E05B
:1019F0000020704700201849096811F0200F01D01D
:101A0000012000E00020704729B1134A1269024307
:101A1000114B1A6104E0104A126982430E4B1A619D
:101A2000704701460020012908D10B4AD26912F003
:101A3000010F01D0012008E0002006E0064AD2682C
:101A40000A4201D0012000E0002070470249C8602E
:101A50007047000000F8FF1F002002402301674587
:101A6000AB89EFCD70470B4880470B4981F308885D
:101A70000A480047FEE7FEE7FEE7FEE7FEE7FEE76F
:101A8000FEE7FEE7FEE7FEE705480649064A074B84
:101A900070470000651A0008980600203101000810
:101AA000980000209806002098020020980200204C
:101AB000704770477047754600F028F8AE4605003D
:101AC0006946534620F00700854618B020B5FFF759
:101AD000DBFFBDE820404FF000064FF000074FF05D
:101AE00000084FF0000B21F00701AC46ACE8C0093C
:101AF000ACE8C009ACE8C009ACE8C0098D46704745
:101B00000446AFF300802046FEF75BFB00487047B9
:101B10003400002003494FF01800ABBE70470000AE
:101B200009000000260002007047000010B591EA8D
:101B3000030F48BF83F0004300F15083841A71EB18
:101B4000030E05D2121943EB0E03001B61EB0E01CD
:101B5000DFF880C14FEA1154A4EB135E1CEA430F77
:101B600018BF9CEA445F7DD023EA0C0321EA0451AC
:101B700043F48013DEF1200C38D322FA0EFC10EB74
:101B80000C0023FA0EFC41EB0C01CEF1200C03FA01
:101B90000CFC10EB0C0051F10001B1F5801FCEF1EF
:101BA000200C38D201EB0451BDE8104012FA0CF2BF
:101BB00058BF7047401C38BF5FEA420218BF7047E9
:101BC000002814BF20F0010041F100014FEA410359
:101BD00013F5001F38BF704728BFB1F1C0413E491F
:101BE0004FF0000048BF41F000417047012A43EB2D
:101BF0000302AEF1200EDEF11F0C32BF4FF0000CDD
:101C000023FA0EF310EB030041EB0451B4EB115F28
:101C1000CAD0A1EB045101F58011490801EB045130
:101C2000BDE810405FEA30000CD350F1000038BF2F
:101C300012FA0CFC06D1C3E7401C38BF5FEA42022F
:101C4000C4D1BDE74FEA410313F5001F38BF704709
:101C500028BFB1F1C04120494FF0000048BF41F01A
:101C6000004170479CEA445F08D0BDE8104011EA8B
:101C70005C0F04BF01F0004100207047012841EBD8
:101C80000104012A43EB030E644598BFE645DFF8E3
:101C90004CC0BDE8104000F22580AFF30080012861
:101CA00041EB0100012A43EB0302904208D010F5FA
:101CB000001F04BF0020704719464FF00000704716
:101CC00091EA030F4FF0000058BF704704494FF0EE
:101CD000000070470000E0FF0000F07F11000004EA
:101CE0000000F87F02494FF0000000F009BC00003E
:101CF0000000F87F02494FF0000000F001BC000036
:101D00000000F87F70B5DFF8ECC33CEA111418BF8F
:101D10003CEA131400F09B8081EA03050CEA1114DD
:101D200044EAD5741CEA131518BF11EA0C1F00F021
:101D300074804FEAC1214FEAC32341EA505143EA7C
:101D40005253A4EB050404F17F7441F0004143F0C9
:101D500000434FEAC0204FEAC22200F0A9F846052E
:101D60004FEAD02003EB244340EA41504FEAD1210F
:101D700001EB035282EAC47116D05FEA460E38BF07
:101D80004FF0404610D314BF00234FF0004350F1F2
:101D9000000041F1000110EAD37F4FF0804620EAB5
:101DA000D37018BF4FF0404691EAC47FDFF848E394
:101DB00016D412EA0E0F18BF3EEA010E10D070BD05
:101DC000E50754BF1EF4000F1EF4800F0ABF4FF04A
:101DD00080464FF0404610F1010041F10001E3E779
:101DE000B4F1806FDEBF01F1C04101F0004100207D
:101DF00000DC70BDA8BFA1F1C04146F0140CA8BF23
:101E00004CF0805CBDE870406FF0000041EA50018A
:101E100081EA10314FF00000704711EA0C1F00D02A
:101E20000AE013EA0C1F00F03D804FF0000081EA49
:101E3000030101F0004170BD6FF0000081EA030171
:101E400041EA500181EA10314FF0000070BD4FEAC5
:101E5000410EBEEB4C1F4FEA430508BF002898BF58
:101E6000B5EB4C1F08BF002ABDE87040DFF88CC2FC
:101E70003FF638AFAFF300804FF4001C1CEB410F6E
:101E800009D11CEB430F0FD04B4021F0004148BF5C
:101E900041F0004170474FF0000081EA030303F076
:101EA00000417047BDE870404FF000009449704712
:101EB000E0B5054610B40C460FF238114FEA430C5A
:101EC0004FF0010E4FEA9C6C51F82CC04FF000010E
:101ED000ACFB02604FF00006ECFB0301001841EB85
:101EE0000101301A66EB0101E1FB0C6C4FF00001BF
:101EF000ACFB02604FF00006ECFB0301001841EB65
:101F00000101301A66EB0101E1FB0C6C4FF000019E
:101F1000ACFB0560ECFB0401A2FB0167E3FB006E78
:101F200017EB0E074FF0000EE3FB017E4EF1000EA3
:101F3000B6197F414EEB0E0E764275EB070764EB48
:101F40000E0EECFB0E01ACFB07E64FF0000E801905
:101F500041F10001A2FB0067B619E2FB017EE3FB41
:101F6000007E7F4103FB01EE4EEB0E0E76424FF0FA
:101F7000000676EB070765EB0E0EACFB0E674FF025
:101F8000000E4FEA857C4FEA9505C01941F100012A
:101F900045EA847549084FEA3000A2FB00677642A3
:101FA000E2FB017EE3FB007E7CEB070703FB01EE17
:101FB00065EB0E0EB51A77EB03047EF1000E24BF1D
:101FC0002E46274650F1000041F10001012E38BF96
:101FD000012F404141EB010111F0004F18BF0223D6
:101FE00001D0F0BC00BDF0BC4FF00103001841EB84
:101FF000010100BDFCC00FFC830F3EF85F8D89F42A
:10200000F0F0F0F0B50373EDEAA00EEA48B4C2E6D2
:10201000E3388EE31C3870E0A6C867DDA70D74DADC
:10202000E53594D7037BC7D4D2200DD2A87464CFF2
:10203000CCCCCCCCE68745CA7C0CCEC77BC865C56A
:10204000C3300CC3C0C0C0C00BFA82BE0B6452BC0C
:10205000A28B2EBAE00217B8B6600BB6B4400BB430
:10206000C84216B2020B2CB05C414CAE849176ACE7
:10207000AAAAAAAA573FE8A839052FA702B57EA5A4
:102080003D0AD7A32BC337A2A0A0A0A0E765119F4C
:102090009DD8899D9CC0099CD9E7909A511A1F9997
:1020A000ED25B4976CDA4F964F09F294C4859A9354
:1020B0009224499209BCFD90EE23B88F6D35788E3D
:1020C00008CB3D8D8CC0088CFBF2D88A8940AE8944
:1020D000888888885FAB67877D8A4B8653083485FC
:1020E00042082184976E12838220088208040281AC
:1020F000000000800000FF070000F07F14000004D3
:102100000000F87F4FEAC12303B40A1543EA505395
:1021100018BF43F000430DD4A2F56072D2F19E02C5
:1021200040F32180FF2ACCBF002123FA02F10846A8
:1021300002B070474FEA4252520D08BF23F00043ED
:102140004FF00001A2F56072D2F19E020BDBFF2A74
:10215000DCBF23FA02FCA1EB0C010029DEBF02B0B8
:1021600008467047FFE703BCDFF830C0012841EBA9
:10217000010313F5001F88BF4CF4803C3FF6BAAD55
:102180003EBF6FEAE17080F000407047AFF300801F
:102190006FEAE17080F0004070470000C800020460
:1021A00010F0004314BF4142014643F08043B1FAAE
:1021B00081FC03F1F87311FA0CF1A3EB0C534FEA15
:1021C000415008BF704703EBE121704710B591EA19
:1021D000030F48BF83F000433FF5B0AC841A71EBA6
:1021E000030E07D212198EF0004E43EB0E03001BB4
:1021F00061EB0E01DFF810C24FEA1154A4EB135E3D
:102200001CEA430F18BF9CEA445F00F0C58023EA34
:102210006C03524221EA0451C3EB6C0338BF5B1ECE
:10222000DEF1200C29D322FA0EFC10EB0C0043FA4D
:102230000EFC41EB0C01CEF1200C03FA0CFC10EB70
:102240000C0051F10001CEF1200C2DD401EB045112
:10225000BDE8104012FA0CF24FF0120C4CF0804C1A
:1022600058BF7047401C1CBFB2F1004F7047002898
:102270000CBF491C20F00100704712EB020C43EB2D
:10228000030218BF4FF0010C4CEA4202AEF1200EDF
:10229000DEF11E0C63D943FA0EFC10EB0C0051F179
:1022A000FF31CEF11E0CD1D50CF1010C12FA0CFC51
:1022B000404141EB010101EB445E5FEA5E5E10D9F3
:1022C00001EB0451BDE8104010EBDC7038BFBCF1ED
:1022D000004F18BF704700280CBF491C20F00100B8
:1022E00070473FD211F5001108BF002801D1BDE8A9
:1022F00010403FD04FEAD42E24F40064B1FA81F2AA
:10230000202AA4F1020404BFB0FA80F3D218A2F18B
:102310000B02B2F12003A4EB02040CD2C2F12003A1
:1023200001FA02F120FA03F341EA030100FA02F094
:10233000C2F1200303E000FA03F14FF0000001EBCB
:10234000CE71002C01EB0451BDE81040A8BF7047CE
:1023500001F1C0414FF0000001F00041704701EB76
:10236000045110BD491001EB0451BDE810404FEA83
:10237000300002E04FF0000170474FF0120C4A00AD
:1023800008BF0042F6D0B2F5001F28BF704701F029
:1023900000414FF0000070479CEA445F07D0BDE861
:1023A000104011EA5C0F04BF002100207047012893
:1023B00041EB0104012A43EB030E644598BFE64557
:1023C000DFF848C0BDE810403FF68CACAFF30080AA
:1023D000012841EB0100012A43EB0302904209D09E
:1023E00010F5001F04BF0020704783F000414FF03C
:1023F0000000704791EA030F4FF0000048BF70479C
:1024000003494FF0000070470000E0FF1200000495
:102410000000F87F094248BF4CF4803C4FF4C06391
:102420004FEA115203F1010321EA025122F4006242
:102430009A1A48BF6FF0FE0241F48011352A3CD849
:1024400030D0152A1ED3203A0CD90028C2F120031F
:1024500021FA02F001FA03F218BF42F001024FF034
:10246000000130E0C2F1000302F1200201FA03F1A1
:1024700020FA02F241EA020100FA03F208464FF0A4
:10248000000120E0C2F1200310B400FA03F401FAC5
:1024900003F320FA02F021FA02F1224610BC43EACB
:1024A000000010E050EA01324FF000004FF0000150
:1024B0004FF0004218BF521C05E04FF001024FF0F0
:1024C00000014FF000001CF4803F2CF4803C18BF4A
:1024D00041F00041124208BF7047520003D303D0BD
:1024E000401C41F1000170475FEAAC72F8D4FAD1A8
:1024F000401C41F1000120F00100F4E770477047F3
:102500000CF00F03092B08BF082000F02B800A2BCA
:102510000BD0082B18BF704708BF1CF0400F0AD023
:102520004FF000004FF0000170471CF0400F18BF43
:102530004FF0004070471CF0100F08D020F070439F
:1025400000F07F4242EAD3014FEA4370704700F047
:10255000604021F07F4242EA000201F07F4040EA01
:10256000727070471CF4801F11D01CF4E02F03D050
:102570006FEACC31490070474FF04050EFF30082D2
:1025800022F0704242EA000282F3008870474FF066
:1025900000007047B425000800000020280000005B
:1025A0006C010008DC2500082800002070060000EF
:1025B000880100080000000000000000000000008A
:1025C0000000000000000000000000000102030401
:0C25D000010203040607080902040608C3
:0400000508000131BD
:00000001FF
